:100000000C942A000C9445000C9445000C94450077
:100010000C9445000C9445000C9445000C9445004C
:100020000C9445000C9445000C9445000C9445003C
:100030000C9445000C9445000C9445000C9445002C
:100040000C9445000C9445000C9445000C9445001C
:100050000C94450011241FBECFE5D8E0DEBFCDBF14
:1000600010E0A0E6B0E0EAE0F1E002C005900D92F9
:10007000A036B107D9F710E0A0E6B0E001C01D92AC
:10008000A036B107E1F70C9455000C9400001CBE9B
:1000900013BC89E683BF85BD0895877087B9369AFA
:1000A0003699FECF84B195B10895CFE5D8E0DEBF93
:1000B000CDBF8FEF87BB81BB84E886B90E94470024
:1000C00010C095958795959587958CBF81E090E0B8
:1000D0000E944D0097FD17C095958795959587953A
:1000E00083BD80E090E00E944D0097FFEACF039629
:1000F00095958795959587958CBF81E090E00E94B6
:0A0100004D0097FFE9CF0396E7CF0B
:00000001FF
